:100000000C9407040C9424040C9424040C942404ED
:100010000C9424040C9424040C9424040C942404C0
:100020000C9424040C9424040C94BF0D0C9424040C
:100030000C9424040C94EC200C9424040C941921AA
:100040000C9424040C9424040C9424040C94240490
:100050000C9424042C2064656743002C20003A0093
:100060003A0054797065202268656C702220666FB2
:100070007220636F6D6D616E64206C6973742E0005
:10008000232073656C66746573742072656164798E
:1000900000232073746172742073656C66746573D9
:1000A000740031303A34323A3530002320536F66D1
:1000B00074776172652054696D65203A200041753E
:1000C000672032362032303039002320536F667477
:1000D000776172652044617465203A2000232050C6
:1000E0004342502D5265666C6F7720436F6E747279
:1000F0006F6C6C65720048656174696E6700556E5F
:100100006B6E6F776E004F6666004175746F6D6140
:10011000746963004D616E75656C6C204F6E004CA8
:100120006561726E004C6561726E205265666C6F1F
:10013000772054656D700000234D6F6465203A2070
:100140000023536574696E672054656D70206F6677
:100150006673657400234572726F722054656D700A
:10016000206469666620746F6F2068696768002084
:1001700064656743290020280020202054203D206A
:10018000200029202020546F6C64203D2020002076
:10019000280020202054203D2020004454203D20D1
:1001A000004F76657273686F6F74203D200000C445
:1001B000079B05000002060738060926060DBA0748
:1001C000001406010000000181077E0739091E06A0
:1001D00000E9050200000102180A7B0723091E0638
:1001E00000E9050300000203DB0978077E091E060B
:1001F00000E90504AE050400000304A909750768B9
:10020000091E0600E9050500000405940972075A55
:10021000091E0600DE0500000005069C059D059EE2
:1002200005000006079F050000A0050C0600000061
:1002300007085F060000A1051E06000000080995DA
:10024000086F074F09420600C8050A0000090A8026
:10025000086C076706420600BD050B00000A0B5339
:10026000086907D60A420600D3050C00000B0C41B2
:10027000086607CC08420600A2050000000C0DAE7F
:100280000863074A0A30060000000D205472616EB0
:1002900073203A20002000205374617465203A20B6
:1002A0000068656C700068696C6665006B657973E1
:1002B0000074656D7073686F770074656D700064AD
:1002C0006562756700747261636500736574746953
:1002D0006E67730070687474656D70007068747414
:1002E000696D650070687470777200736F616B740C
:1002F000656D7000736F616B74696D6500736F611C
:100300006B707772007265666C6F7774656D7000E4
:100310007265666C6F7774696D65007265666C6F87
:1003200077707772006477656C6C74656D700064CB
:1003300077656C6C74696D65006477656C6C70775B
:10034000720074656D706F6666736574004C6973D6
:1003500074657420616C6C652042656665686C65C7
:10036000206175660054617374656E66756E6B749A
:10037000696F6E656E0054656D706572617475723B
:10038000206A6564652053656B756E6465206175D0
:1003900073676562656E205B506172616D6574653F
:1003A000722030206F64657220315D0054656D707D
:1003B0006572617475722065696E6D616C20616E25
:1003C0007A656967656E00446562756767696E671F
:1003D00020496E666F726D6174696F6E656E202064
:1003E000617573676562656E2020205B5061726184
:1003F0006D657465722030206F64657220315D0018
:10040000496E7465726E65204175746F6D617465B7
:100410006E7A75737461656E646520617573676566
:1004200062656E205B506172616D6574657220302B
:10043000206F64657220315D00416C6C65204569F8
:100440006E7374656C6C756E67656E20617573672D
:100450006562656E00507265686561742054656DF3
:10046000706572617475725B302E2E3235345D208A
:10047000477261640050726568656174205A6569ED
:10048000742020202020205B302E2E3235345D2039
:1004900053656B0050726568656174204C656973C3
:1004A00074756E672020205B302E2E3130305D2039
:1004B0002500536F616B2054656D706572617475B2
:1004C0007220205B302E2E3235345D2047726164FD
:1004D00000536F616B205A65697420202020202012
:1004E00020205B302E2E3235345D2053656B005357
:1004F0006F616B204C65697374756E6720202020D6
:10050000205B302E2E3130305D2025005265666C28
:100510006F772054656D70657261747572205B3001
:100520002E2E3235345D2047726164005265666C50
:100530006F77205A656974202020202020205B30AE
:100540002E2E3235345D2053656B005265666C6F1C
:1005500077204C65697374756E67202020205B30AE
:100560002E2E3130305D2025004477656C6C205490
:10057000656D70657261747572205B302E2E323538
:10058000345D2047726164004477656C6C205A6565
:100590006974202020202020205B302E2E3235341C
:1005A0005D2053656B004477656C6C204C65697306
:1005B00074756E67202020205B302E2E3130305D28
:1005C00020250054656D70657261747572204A75DE
:1005D0007374616765205B2D33302E2E33305D20C0
:1005E000477261640054617374656E203A0D0A317C
:1005F000203D20417573736368616C74656E0D0AEC
:1006000032203D204175746F6D6174697363686554
:1006100072204C6F6574626574726965620D0A338D
:10062000203D204F66656E706172616D6574657204
:10063000204C65726E656E0D0A000D0A4175746F6F
:100640006D6174697363686572204C6F657462656F
:100650007472696562206E6F6368206E6963687486
:10066000206D6F65676C6963682E0D0A426974744A
:10067000652065727374204F66656E706172616D7E
:10068000657465722065696E6C65726E656E0D0AC3
:100690000000A1024D0300C81C000000AC0265036D
:1006A00000B21C000000A6024D0300C81C000000A0
:1006B000CB023904007519000000D402550400096A
:1006C0001CFC1700DC02750400E01B051800E402A6
:1006D000940400B71B171800EB02B204008E1B58DD
:1006E0001800F402D10400651B611800FD02EF043C
:1006F000003C1B73180005030C0500131B101900A8
:1007000010032C0500EA1A1919001B034B0500C140
:100710001A2B19002503690500981AB418002F0335
:100720008805006F1ABD18003903A60500461ACFC8
:1007300018004203C30501111A000000B10276033C
:10074000019B1C000000BA02AC0300321C00000038
:10075000BF02C70300791C000000C5020004005757
:100760001C0000000000000000000000002020200D
:1007700000203D200020202000203D200020646536
:1007800067430054656D70203A2000232054726145
:100790006365204F46460023205472616365204FF5
:1007A0004E0023204465627567204F464600232093
:1007B0004465627567204F4E00232054656D707349
:1007C000686F77204F464600203A200023202043C0
:1007D0006F6D6D616E6473203A2000232075736520
:1007E000202268656C7022002320436F6D6D616E5E
:1007F00064206E6F7420666F756E64003031323322
:1008000034353637383941424344454600001124D7
:100810001FBECFE5D8E0DEBFCDBF10E0A0E6B0E060
:10082000EEEBFAE402C005900D92AA3BB107D9F7AE
:1008300012E0AAEBB0E001C01D92A238B107E1F7C7
:100840000E9426040C945D250C9400002F923F9288
:100850004F925F926F927F928F929F92AF92BF92D0
:10086000CF92DF92EF92FF920F931F93DF93CF937C
:1008700000D000D00F92CDB7DEB7A79AAF988FEB1C
:1008800087BB88B38F6B88BBC098C79A0E94500CF7
:100890000E94FA100E9437100E94D21D0E949B21D4
:1008A0000E946C19789460E875E280E090E00E9404
:1008B0009C2089EC90E20E94941F8DED90E00E94B4
:1008C000B11F0E94C81F8AEC90E00E94B11F8EEBFE
:1008D00090E00E94B11F0E94C81F8BEA90E00E9426
:1008E000B11F82EA90E00E94B11F0E94C81F0E94BF
:1008F00048150E94D40781E065E370E040E80E945B
:100900007B1F80E00E94271F81E990E00E94B11FB9
:100910000E94C81F08E119E70DC0C09AC8010197DD
:10092000F1F7C8010197F1F7C8010197F1F7C80184
:100930000197F1F780E00E94DA1D8F5F9F4F31F43D
:100940000E940910882349F7C098E8CFC09A1982FD
:10095000AA2401E010E004C0AA2489818930D1F0E2
:100960000E9409108823C1F3AA2089F488B38F6BF1
:1009700088BB38B32981C801022E02C0880F991F95
:100980000A94E2F78095832388BB2F5F2983AA24EA
:10099000A394E3CF88B38F6B88BB80E890E00E947C
:1009A000B11F0E94C81F82E690E00E94B11F0E9402
:1009B000C81F0E942A10AC01CB01DA017C018D0115
:1009C0001E010894211C311C0E94E517882339F56B
:1009D0000E942A100E94F4070E941D1180E00E94CC
:1009E000D2108823E1F581E00E94D210882399F586
:1009F00082E00E94D210882351F5C1010E946E212D
:100A0000882309F50E94CE178F3FF1F60E94091046
:100A1000882379F1C4980E94E5178823C9F20E94BF
:100A20002A106A837B838C839D83E616F70608076A
:100A3000190729F1AA2029F1EA80FB800C811D8188
:100A4000AA24A394C5CF89810E948B1DDBCF84E0AB
:100A50000E944A06D2CF81E00E944A06C9CF0E9476
:100A60004F06843041F00E94B20F82E00E944A0695
:100A7000BACFC49AA9CF85E00E944A06B4CFAA246F
:100A8000A7CF6A817B818C819D810E94660BE72EB6
:100A9000A82E692E80E00E94DA1D582E492EFF24D0
:100AA00000E010E08AE062E040E020E30E94D51F11
:100AB00080E690E00E94B11FBB24CC24DD248AE0B4
:100AC00062E040E020E3860175010E94D51F8EE5BB
:100AD00090E00E94B11F7724882499248AE062E084
:100AE00040E020E3840173010E94D51F8BE590E074
:100AF0000E94B11F252D342DC90197FD16C0959573
:100B00008795959587957C010027F7FC0095102F18
:100B10008AE064E041E020E30E94D51F84E590E094
:100B20000E94B11F0E94C81F87CF0396E8CF81E0C3
:100B30008093D40008950895089508950895089520
:100B40000895089520E0809112029091130297FD7C
:100B500002C0822F089521E0822F089540E0209165
:100B6000D9003091DA008091DB009091DC002817E9
:100B700039070CF041E0842F089520E08091D900DE
:100B80009091DA00883C91050CF021E0822F0895C5
:100B900020E08091D9009091DA00893C91050CF415
:100BA00021E0822F089520E08091D9009091DA0011
:100BB000805991400CF021E0822F089520E080912F
:100BC000D9009091DA00815491400CF421E0822FF9
:100BD000089560E02091C3003091C4004091C500A9
:100BE0005091C6008091C7009091C800A091C900A3
:100BF000B091CA00281739074A075B0708F061E07F
:100C0000862F089590E08091BD00833011F0892FE8
:100C1000089591E0892F089590E08091BD00833080
:100C200009F091E0892F089590E08091BD00823015
:100C300011F0892F089591E0892F089590E0809117
:100C4000BD00823009F091E0892F089590E08091F5
:100C5000BD00853011F0892F089591E0892F089506
:100C600090E08091BD00853009F091E0892F0895D2
:100C700090E08091BD00843011F0892F089591E0BB
:100C8000892F089590E08091BD00843009F091E0B3
:100C9000892F0895863010F48093BE0008958091C6
:100CA000BD0008951F93182F0E948917882329F0EB
:100CB0008091DD00612F0E9446141F91089588EBFA
:100CC0009BE068E370E040E80E94050B0895809186
:100CD000D5009091D6000E94AE0D1092D3000E94D4
:100CE000401F0895EF92FF920F931F938091BA00D7
:100CF0009091BB00892B09F444C00E9409108823FD
:100D000079F18091BC00882309F047C0E091D900B7
:100D1000F091DA008091140290E02091120230915B
:100D20001302AC01429FC001439F900D529F900D52
:100D3000112464E670E00E94D624E60FF71F80912C
:100D4000D7009091D800E817F90794F081E08093DC
:100D5000D3000E94401F1F910F91FF90EF900895C4
:100D60008091BC00882391F681E08093BC00CECFB7
:100D70001092D3000E944E1F1F910F91FF90EF9091
:100D8000089580E00E94DA1D9093DA008093D900E4
:100D90009093BB008093BA00B0CF80E00E94DA1D30
:100DA0009093DA008093D9002091BA003091BB0073
:100DB000821B930BAC01440F551F480F591F440F62
:100DC000551F440F551F440F551F480F591F2091A1
:100DD000120230911302C901880F991F820F931FCD
:100DE000480F591F57FD6AC055954795559547952A
:100DF00050931302409312021092BC000E94A0175D
:100E0000882349F4E091D900F091DA00F093BB0017
:100E1000E093BA007FCF8BE991E00E94B11FE09090
:100E20001202F09013020027F7FC0095102F8AE0C1
:100E300064E041E020E20E94D51F82E991E00E9437
:100E4000B11FE090D900F090DA000027F7FC009580
:100E5000102F8AE064E041E020E20E94D51F8FE875
:100E600091E00E94B11F2091D9003091DA00C901B0
:100E700097FD27C095958795959587957C010027C7
:100E8000F7FC0095102F8AE064E041E020E20E9428
:100E9000D51F82E891E00E94B11FE090BA00F09067
:100EA000BB000027F7FC0095102F8AE064E041E0CA
:100EB00020E20E94D51F0E94C81FA4CF4D5F5F4F44
:100EC00093CF0396D7CF0E94720608950E947206B0
:100ED00008950E94720608950E94720608950E9465
:100EE000720608950E94720608950E94720608957F
:100EF0000E94720608950E94720608950E9472066A
:100F000008950E9417180E94271F0E94051820911B
:100F1000C3003091C4004091C5005091C600280F15
:100F2000311D411D511D2093C7003093C8004093CF
:100F3000C9005093CA000E94FC1790E0880F991FC7
:100F4000880F991F9093D8008093D700C0980E9473
:100F50008317BC0187E995E00E94170D9093D60096
:100F60008093D50088EE93E068E370E040E80E944B
:100F7000050B08950E94CE1790E08F3F11F0892F46
:100F8000089591E0892F08950E94401F88B38F61D2
:100F900088BBC79A0E94CE17809314028F3F09F036
:100FA00008951092140208951092D4001092D30064
:100FB00081E08093BD008093BE0080E690E06DEDFF
:100FC00070E046EF50E00E94F7129093C0008093CB
:100FD000BF000E948917882309F408958091DD00DD
:100FE00060E00E94461408956093C3007093C400AB
:100FF0008093C5009093C6008091BF009091C0007F
:101000009093C2008093C10060E670E04DED50E027
:101010000E941C129093C0008093BF002091C100D9
:101020003091C2008217930721F00E94891788230C
:1010300069F49091BE008091BD00891731F09093C2
:10104000BD000E94A017882339F408958091DD0027
:1010500060E00E944614EDCF88E391E00E94B11F4A
:101060008091BD0090E0FC01EE0FFF1FE80FF91F1B
:10107000E456FF4F818192810E94B11F0E94C81FD8
:10108000089588E290E09093D8008093D7000E9462
:101090008317BC0187E995E00E94170D9093D60055
:1010A0008093D500089510921302109212021092AC
:1010B0001102109210028091C3009091C400A0917F
:1010C000C500B091C6008093CB009093CC00A09354
:1010D000CD00B093CE0088E092E09093D80080934A
:1010E000D7000E948317BC0187E995E00E94170D85
:1010F0009093D6008093D50084E60E94271F089520
:1011000088E092E09093D8008093D7000E948317E4
:10111000BC0187E995E00E94170D9093D60080935B
:10112000D50084E60E94271F08950E94401F88B3BF
:101130008F6088BBC79AC49888E290E09093D800EB
:101140008093D7000E948317BC0187E995E00E9435
:10115000170D9093D6008093D500089584E60E94E1
:10116000271F80EB94E09093D8008093D700C49819
:10117000C0980E948317BC0187E995E00E94170D73
:101180009093D6008093D50088EE93E068E370E0FA
:1011900040E80E94050B0895EF92FF920F931F9372
:1011A0006091D9007091DA00882777FD8095982F9B
:1011B00029E130E040E050E00E94A32460517742F2
:1011C000804090402091100230911102442737FD59
:1011D0004095542F0E940B25209314020E94A017C3
:1011E000882389F081EA91E00E94B11FE090140207
:1011F000FF2400E010E08AE064E041E020E20E9489
:10120000D51F0E94C81F8091D5009091D6000E94E2
:10121000AE0D1092D3000E94401FC49A88EE93E056
:1012200068E370E040E80E94050B809114020E9480
:10123000D71781E08093BD008093BE001F910F916E
:10124000FF90EF90089580E00E94271F8091D500C5
:101250009091D6000E94AE0D1092D3000E94401FC4
:10126000C19A84E690E068E370E040E80E94050BD4
:10127000089580E00E94271FC09A8091D500909128
:10128000D6000E94AE0D1092D3000E94401F84E64B
:1012900090E068E370E040E80E94050B08958091BB
:1012A000D5009091D6000E94AE0D1092D3000E94FE
:1012B000401F089581E08093BE008091D5009091F9
:1012C000D6000E94AE0D1092D3000E94401F0895D8
:1012D00080E00E94271F8091D5009091D6000E9447
:1012E000AE0D1092D3000E94401FC39A80EA9FE087
:1012F00068E370E040E80E94050B089580E00E94DA
:10130000271F8091D5009091D6000E94AE0D1092BB
:10131000D3000E94401FC29A84E690E068E370E028
:1013200040E80E94050B089580E00E94271F88EC8A
:1013300090E09093D8008093D7000E948317BC015F
:1013400087E995E00E94170D9093D6008093D50011
:1013500008950E94CF180E94271F0E94BD18209157
:10136000C3003091C4004091C5005091C600280FC1
:10137000311D411D511D2093C7003093C80040937B
:10138000C9005093CA000E94B41890E0880F991FBA
:10139000880F991F9093D8008093D7000E948317DD
:1013A000BC0187E995E00E94170D9093D6008093C9
:1013B000D500C39808950E942B190E94271F0E94F0
:1013C00019192091C3003091C4004091C50050917B
:1013D000C600280F311D411D511D2093C7003093B9
:1013E000C8004093C9005093CA000E94101990E0B1
:1013F000880F991F880F991F9093D8008093D7006A
:101400000E94101990E0880F991F880F991F9093E0
:10141000DC008093DB000E948317BC0187E995E024
:101420000E94170D9093D6008093D500C29808951E
:101430000E9473180E94271F0E9461182091C30008
:101440003091C4004091C5005091C600280F311D55
:10145000411D511D2093C7003093C8004093C9001F
:101460005093CA000E94581890E0880F991F880F67
:10147000991F9093D8008093D7000E948317BC01D6
:1014800087E995E00E94170D9093D6008093D500D0
:10149000C1980895EF92FF920F931F93CF93DF931C
:1014A0000E94401FC49AC09A0E94A017882309F086
:1014B00048C08091D5009091D6000E94AE0D109248
:1014C000D3000E94401F81E08093BD008093BE0046
:1014D0000E941019C82FD0E0CC0FDD1FCC0FDD1FEC
:1014E0008091D9009091DA00C81BD90BCE018258A7
:1014F0009F4F8D3F9105D8F48C2F0E94C01781E437
:1015000091E00E94B11F7E010027F7FC0095102F8B
:101510008AE064E041E020E20E94D51F0E94C81FDB
:10152000DF91CF911F910F91FF90EF90089588EB7D
:101530009BE068E370E040E80E94050B85E591E0E0
:10154000E0CF89E791E00E94B11FE090D900F090D0
:10155000DA000027F7FC0095102F8AE064E041E0F4
:1015600020E20E94D51F86E791E00E94B11F2091E2
:10157000D9003091DA00C90197FD16C0959587957D
:10158000959587957C010027F7FC0095102F8AE040
:1015900064E041E020E20E94D51F8FE691E00E94C6
:1015A000B11F0E94C81F85CF0396E8CF8091D50058
:1015B0009091D6000E94AE0D1092D3000E94401F61
:1015C0008091C3009091C400A091C500B091C60065
:1015D0008093CF009093D000A093D100B093D2001D
:1015E0008091120290911302909311028093100245
:1015F0000E94401F0895E0911502F091160280812B
:1016000090911702892B808308959C017093160294
:1016100060931502409317028233910510F422E380
:1016200030E08BEF9AE0B9010E94810CE091150245
:10163000F091160290818091170280958923808312
:101640000895BF92CF92DF92EF92FF920F931F9374
:10165000262FC72EE82EB92E30E040E050E0CA0118
:10166000B90120E831E541E050E00E94A3249B014C
:10167000AC012B0D311D411D511DDD2480E19EE08B
:10168000BC01C69EC001C79E900DD69E900D112430
:10169000AA2797FDA095BA2F280F391F4A1F5B1F55
:1016A0008CE3E89E700111240027F7FC0095102FB1
:1016B0002E0D3F1D401F511FB901CA011F910F91EF
:1016C000FF90EF90DF90CF90BF9008959F92AF92E0
:1016D000BF92CF92DF92EF92FF920F931F935B0125
:1016E0006C0160304CE8740749E0840740E09407DF
:1016F00008F04EC020E831E541E050E00E94E924C6
:10170000922E622F70E080E090E020E83EEA4EEFFB
:101710005FEF0E94A3247B018C01EA0CFB1C0C1DD3
:101720001D1DC801B70120E13EE040E050E00E94ED
:10173000E924D22E30E08CE49EE0AC01249FC0016D
:10174000259F900D349F900D1124AA2797FDA095F9
:10175000BA2FE81AF90A0A0B1B0BC801B7012CE3D0
:1017600030E040E050E00E94E9248CE3289FC00173
:1017700011249E2D981B692D7D2D822F1F910F9175
:10178000FF90EF90DF90CF90BF90AF909F90089523
:1017900097E0992E87E1D82E2BE39BE3ECCF60E80E
:1017A00071E581E090E0089560E17EE080E090E006
:1017B00008956CE370E080E090E0089561E070E0EF
:1017C00080E090E00895EF92FF920F931F937B01CA
:1017D0008C01E20EF31E041F151F80E0E8168CE852
:1017E000F80689E0080780E01807D0F01216130603
:1017F00014061506E4F480E094E7A6EFBFEFE80EC8
:10180000F91E0A1F1B1FC801B70120E03CE849E090
:1018100050E00E94E924AC01CB01DA017C018D018A
:10182000B701C8011F910F91FF90EF90089580E0DC
:101830009CE8A9E0B0E0E80EF91E0A1F1B1F90E02B
:10184000E9169CE8F90699E0090790E0190778F78E
:10185000E7CFEF92FF920F931F93261737074807A2
:10186000590778F079018A01E61AF70A080B190B73
:10187000C801B70180E090E01F910F91FF90EF90B9
:10188000089560507447864F9F4F621B730B840B03
:10189000950B80E090E01F910F91FF90EF900895DD
:1018A0001092DF001092DE001092E6001092E50028
:1018B0001092ED001092EC001092F4001092F300E0
:1018C0001092FB001092FA00109202011092010196
:1018D00010920901109208011092100110920F014C
:1018E000109217011092160110921E0110921D0104
:1018F00087E48CBF83B78D6083BF89B7826089BF5F
:101900000895CF93DF93EC018091DE009091DF008A
:10191000892B09F445C08091E5009091E600892B60
:1019200009F46AC08091EC009091ED00892B09F4D4
:1019300066C08091F3009091F400892B09F462C095
:101940008091FA009091FB00892B09F45EC0809190
:10195000010190910201892B09F45AC0809108017C
:1019600090910901892B09F456C080910F01909143
:101970001001892B09F452C0809116019091170132
:10198000892B09F44EC080911D0190911E01892B75
:1019900009F44AC02FEF3FEFC901DF91CF910895BD
:1019A00080E090E09C01FC01EE0FFF1FEE0FFF1F97
:1019B000EE0FFF1FE21BF30BE252FF4F1682138262
:1019C0001282CB0105966AE070E00E94C224758302
:1019D0006483F894F901EE0FFF1FEE0FFF1FEE0F67
:1019E000FF1FE21BF30BE252FF4FD183C0837894B9
:1019F000C901DF91CF91089581E090E0D3CF82E0DB
:101A000090E0D0CF83E090E0CDCF84E090E0CACFEB
:101A100085E090E0C7CF86E090E0C4CF87E090E01B
:101A2000C1CF88E090E0BECF89E090E0BBCFCF93FC
:101A3000DF93EC018091DE009091DF00892B09F4A7
:101A400045C08091E5009091E600892B09F46BC0B8
:101A50008091EC009091ED00892B09F467C0809192
:101A6000F3009091F400892B09F463C08091FA008F
:101A70009091FB00892B09F45FC080910101909146
:101A80000201892B09F45BC0809108019091090142
:101A9000892B09F457C080910F0190911001892B77
:101AA00009F453C08091160190911701892B09F414
:101AB0004FC080911D0190911E01892B09F44BC0EC
:101AC0002FEF3FEFC901DF91CF91089580E090E0C3
:101AD0009C01FC01EE0FFF1FEE0FFF1FEE0FFF1F1B
:101AE000E81BF90BE252FF4F81E0868313821282DA
:101AF000CB0105966AE070E00E94C224758364837E
:101B0000F894F901EE0FFF1FEE0FFF1FEE0FFF1FFE
:101B1000E21BF30BE252FF4FD183C0837894C901DB
:101B2000DF91CF91089581E090E0D2CF82E090E004
:101B3000CFCF83E090E0CCCF84E090E0C9CF85E0C8
:101B400090E0C6CF86E090E0C3CF87E090E0C0CFC2
:101B500088E090E0BDCF89E090E0BACFF894FC0136
:101B6000EE0FFF1FEE0FFF1FEE0FFF1FE81BF90B1D
:101B7000E252FF4F118210827894089508951F92C7
:101B80000F920FB60F9211242F933F934F935F93B1
:101B90006F937F938F939F93AF93BF93EF93FF9335
:101BA0008091DE009091DF00892BA9F08091E00008
:101BB0009091E10001969093E1008093E0002091E4
:101BC000E0003091E1008091E2009091E30028175D
:101BD000390708F003C18091E5009091E600892B58
:101BE000A9F08091E7009091E80001969093E800B9
:101BF0008093E7002091E7003091E8008091E900B0
:101C00009091EA002817390708F06CC18091EC0028
:101C10009091ED00892BA9F08091EE009091EF005A
:101C200001969093EF008093EE002091EE003091AA
:101C3000EF008091F0009091F1002817390708F02B
:101C400043C18091F3009091F400892BA9F0809119
:101C5000F5009091F60001969093F6008093F500C0
:101C60002091F5003091F6008091F7009091F800F6
:101C70002817390708F01AC18091FA009091FB00EB
:101C8000892BA9F08091FC009091FD000196909322
:101C9000FD008093FC002091FC003091FD008091BC
:101CA000FE009091FF002817390708F0F1C08091DD
:101CB000010190910201892BA9F08091030190917B
:101CC0000401019690930401809303012091030184
:101CD0003091040180910501909106012817390780
:101CE00008F0C7C08091080190910901892BA9F0E3
:101CF00080910A0190910B01019690930B018093C2
:101D00000A0120910A0130910B0180910C01909100
:101D10000D012817390708F09DC080910F0190919F
:101D20001001892BA9F08091110190911201019667
:101D300090931201809311012091110130911201B1
:101D400080911301909114012817390708F073C08E
:101D50008091160190911701892BA9F080911801AB
:101D60009091190101969093190180931801209187
:101D700018013091190180911A0190911B012817C7
:101D8000390708F049C080911D0190911E01892BEF
:101D9000A1F080911F019091200101969093200164
:101DA00080931F0120911F0130912001809121011A
:101DB000909122012817390700F5FF91EF91BF910B
:101DC000AF919F918F917F916F915F914F913F91D3
:101DD0002F910F900FBE0F901F901895E091DE008D
:101DE000F091DF0009958091E400882309F4B5C0E3
:101DF0001092E1001092E000EECEE0911D01F09112
:101E00001E01099580912301882309F4A1C0109235
:101E1000200110921F01D1CFE0911601F09117011E
:101E2000099580911C01882309F48DC01092190135
:101E300010921801A8CFE0910F01F09110010995BF
:101E400080911501882309F479C010921201109233
:101E500011017ECFE0910801F0910901099580916F
:101E60000E01882309F465C010920B0110920A013B
:101E700054CFE0910101F091020109958091070191
:101E8000882309F451C010920401109203012ACF53
:101E9000E091FA00F091FB00099580910001882300
:101EA000F1F11092FD001092FC0001CFE091F300DF
:101EB000F091F40009958091F900882359F110926E
:101EC000F6001092F500D8CEE091EC00F091ED0014
:101ED00009958091F2008823C1F01092EF001092D2
:101EE000EE00AFCEE091E500F091E600099580911B
:101EF000EB00882329F01092E8001092E70086CECC
:101F00001092E6001092E50081CE1092ED00109242
:101F1000EC0097CE1092F4001092F300ADCE109228
:101F2000FB001092FA00C3CE109202011092010140
:101F3000D9CE1092090110920801EFCE1092100133
:101F400010920F0105CF10921701109216011BCFAE
:101F500010921E0110921D0130CF1092DF001092DE
:101F6000DE0039CE10922501109226011092270131
:101F70001092280110922C0110922D0110922E0126
:101F800010922F01089590E080912401882309F494
:101F900091E0909324019923D9F180912C019091A3
:101FA0002D01A0912E01B0912F010196A11DB11D0F
:101FB00080932C0190932D01A0932E01B0932F01BB
:101FC00080912901882321F1809125018F5F8093E1
:101FD00025018C33E8F010922501809126018F5F56
:101FE000809326018C33A0F0109226018091270166
:101FF0008F5F80932701883158F0109227018091DC
:1020000028018F5F80932801883010F010922801FA
:102010000895809124010895882321F08091290159
:10202000882319F01092290108951092240181E06B
:1020300080932901F8941DBC1CBC78940895F894F1
:10204000789460912C0170912D0180912E019091D6
:102050002F010895F89490912501809126017091A7
:1020600027017894609128010E94210B0895109215
:10207000250110922601109227011092280110923A
:102080002C0110922D0110922E0110922F0183EC41
:102090009FE064EF71E00E94170D90932B018093F5
:1020A0002A011092240181E080932901F8941DBC3B
:1020B0001CBC7894089581E0809338010895E82F3E
:1020C000F0E0EE0FFF1FE05DFE4F8181817008950B
:1020D000E0913601F09137013196F0933701E093AA
:1020E0003601E330F105A8F1109237011092360164
:1020F00021E030E0E22FF0E0EE0FFF1FE05DFE4F49
:10210000818180FD20C02F5F3F4F2330310510F0CB
:1021100020E030E0E22FF0E0EE0FFF1FE05DFE4F29
:10212000818180FD10C02F5F3F4F2330310510F0BB
:1021300020E030E0E22FF0E0EE0FFF1FE05DFE4F09
:10214000818180FF0FC03093370120933601822FA9
:1021500008959F012F5F3F4F2330310558F220E053
:1021600030E0C8CF309337012093360184E00895E2
:10217000E82FF0E0EE0FFF1FE05DFE4F818190E061
:10218000969587959695879581700895E82FF0E04C
:10219000EE0FFF1FE05DFE4F818190E096958795E1
:1021A00081700895E82FF0E0EE0FFF1FE05DFE4F15
:1021B0002181822F90E09695879596958795982F07
:1021C000917080FF02C02B7F2183892F0895E82F13
:1021D000F0E0EE0FFF1FE05DFE4F2181822F90E0C7
:1021E00096958795982F917080FF02C02D7F21834F
:1021F000892F089581B38F7181BB82B3806E82BBBA
:10220000109230011092310110923201109233017C
:10221000109234011092350110923701109236015C
:10222000109238018BE590E16AE070E00E94170D92
:1022300090933A0180933901089580913801882361
:1022400089F11092380130B337FD7EC080913001A2
:10225000880F81608093300121E090E08F70907052
:10226000009709F10F97F9F036FF29C080913201EC
:10227000880F8093320120E090E08F70907000977B
:1022800051F10F9741F135FF31C080913401880F32
:102290008093340120E090E08F709070009791F16E
:1022A0000F9781F10895222309F446C080913101EE
:1022B00080FF85608D7F8093310136FDD7CF80917F
:1022C0003201880F81608093320121E090E08F70AD
:1022D00090700097B1F6222339F18091330180FF8D
:1022E00085608D7F8093330135FDCFCF80913401A0
:1022F000880F81608093340121E090E08F709070AE
:10230000009771F6222341F08091350180FF8560AE
:102310008D7F8093350108958091350180FD826025
:102320008A7F8093350108958091330180FD82601A
:102330008A7F80933301A7CF8091310180FD826035
:102340008A7F8093310190CF80913001880F8093F4
:10235000300120E082CFDF93CF93CDB7DEB72E9749
:102360000FB6F894DEBF0FBECDBFFC018491898308
:10237000319684918A83319684918B8331968491AE
:102380008C83319684918D83319684918E8331969E
:10239000E491EF83DE011896FE01319687E001900B
:1023A0000D928150E1F7288539854A855B856C85DA
:1023B0007D858E8590E02E960FB6F894DEBF0FBE19
:1023C000CDBFCF91DF910895DF93CF9300D000D0A0
:1023D00000D0CDB7DEB7FC0184918983319684911A
:1023E0008A833196E491EB83DE011496FE013196E7
:1023F00083E001900D928150E1F76C817D818E81A7
:1024000090E026960FB6F894DEBF0FBECDBFCF91F9
:10241000DF91089580E0089580E0089580E00895B8
:1024200082E00E94D210089581E00E94D2100895A7
:1024300080E00E94D21008953F924F925F926F9277
:102440007F928F929F92AF92BF92CF92DF92EF9244
:10245000FF920F931F93DF93CF93CDB7DEB7A29771
:102460000FB6F894DEBF0FBECDBF5C013B012A0161
:10247000FC01028113810190F081E02D84918F8312
:102480003196849188873196849189873196849199
:102490008A87319684918B87319684918C87319687
:1024A000E491ED87DE011E96FE01379687E00190EC
:1024B0000D928150E1F729893A893E848B889C8866
:1024C000F801849189830F5F1F4FF80184918A83FB
:1024D0000F5F1F4FF8018491025010408B83E980F9
:1024E000FA80D82E2115310511F0F9010995E11472
:1024F000F10409F479C0CC24C39418C0C3940D5FCF
:102500001F4FF80184918C830F5F1F4FF801849156
:102510008D830F5F1F4FF8018491025010408E830E
:10252000EC80FD80D82EE114F10421F0F70109952B
:10253000882321F33D1409F455C08114910411F04E
:10254000F40109950D2D10E0000F111F000F111F50
:10255000060D171DD801ED91FC9184918D8B31965C
:1025600084918E8B319684918F8B31968491888F54
:1025700031968491898F319684918A8F3196E49136
:10258000EB8FDE015C96FE01759687E001900D925F
:102590008150E1F7FC8CED8DFE8D309709F00995A7
:1025A0004114510431F0F20180816F2D4C2D0E94B5
:1025B0002314C801A2960FB6F894DEBF0FBECDBF9C
:1025C000CF91DF911F910F91FF90EF90DF90CF900F
:1025D000BF90AF909F908F907F906F905F904F9043
:1025E0003F9008958501E5CFCC24C394A3CFAF924B
:1025F000BF92CF92DF92FF920F931F93DF93CF93FF
:10260000CDB7DEB765970FB6F894DEBF0FBECDBF6E
:102610008C016B015A01DC01ED91FC91849188875A
:10262000319684918987319684918A8731968491F5
:102630008B87319684918C87319684918D873196E2
:10264000E491EE879E01215F3F4FD901FE0138964C
:1026500087E001900D928150E1F7DE011196F901BA
:1026600087E001900D928150E1F7EA81FB81F980CA
:10267000309709F00995C114D10431F08F2DB501BF
:102680000E949A13F6018083C80165960FB6F894EC
:10269000DEBF0FBECDBFCF91DF911F910F91FF9095
:1026A000DF90CF90BF90AF90089510923C011092B0
:1026B0003B011092500110924F0110926401109250
:1026C0006301109278011092770110928C011092A0
:1026D0008B01089580913B0190913C01892B31F150
:1026E00021E0322F3F5F80914F0190915001892B63
:1026F00009F0232F322F3F5F809163019091640195
:10270000892B09F0232F322F3F5F80917701909121
:102710007801892B09F0232F322F3F5F80918B01A5
:1027200090918C01892B21F0832F089520E0D9CF3F
:10273000822F08950F931F93182F6115710511F1C2
:1027400080913B0190913C01892B09F454C0809108
:102750004F0190915001892B09F451C08091630180
:1027600090916401892B09F44EC08091770190917A
:102770007801892B09F44BC080918B0190918C01D9
:10278000892B21F08FEF1F910F91089504E044E011
:1027900050E0DA01AA0FBB1FAA0FBB1F9D01220F39
:1027A000331F220F331F2A0F3B1F255C3E4FF901B9
:1027B00071836083FA01EE0FFF1FCA01880F991F12
:1027C000880F991F880F991FE80FF91FEE0FFF1F41
:1027D000E35CFE4F81E08083F9011382A40FB51FF3
:1027E000AA0FBB1FAA0FBB1FA15CBE4F1C93802F5B
:1027F0001F910F91089500E040E050E0CACF01E042
:1028000041E050E0C6CF02E042E050E0C2CF03E03A
:1028100043E050E0BECF8F3FA9F085309CF4E82F15
:10282000FF27E7FDF095EE0FFF1FEE0FFF1FCF0113
:10283000880F991F880F991FE80FF91FE55CFE4F5D
:10284000118210820895E82F8F3FE1F08530D4F493
:1028500084E1E802D0011124A55CBE4FFD01838113
:10286000E80FF11D44878F5FFD018383883059F0A5
:10287000FD019281983010F49F5F9283FD01E80F73
:10288000F11D64830895138280E0F2CFAF92BF926E
:10289000CF92DF92EF92FF920F931F93DF93CF932C
:1028A000CDB7DEB76E970FB6F894DEBF0FBECDBFC3
:1028B000282F8F3F09F484C085300CF081C0E82FA9
:1028C000FF27E7FDF095EE0FFF1FEE0FFF1FCF0173
:1028D000880F991F880F991FE80FF91FE55CFE4FBD
:1028E00080819181892B09F46BC084E12802600109
:1028F00011248BE391E0C80ED91EF60180819181ED
:102900000E94B11F87E992E00E94B11FF601828107
:10291000883008F466C0F60113811F5F198288238E
:1029200009F461C000E07E010894E11CF11C91EB08
:10293000A92E90E0B92E2EC0A12FB0E01F5F8DB759
:102940009EB708970FB6F8949EBF0FBE8DBF2DB7E8
:102950003EB72F5F3F4FEDB7FEB7F282E182F9013C
:10296000B382A282F582E482AC0DBD1DFD0184819B
:10297000F901868317820E9402220F5F8DB79EB7EE
:1029800008960FB6F8949EBF0FBE8DBFF6018281E8
:10299000081768F5183081F6A0E0B0E011E0CFCF5D
:1029A0000E94C81FF601808191810E94B11F8BE8AF
:1029B00092E00E94B11FC7010E949F1F0E94C81F82
:1029C0006E960FB6F894DEBF0FBECDBFCF91DF91EC
:1029D0001F910F91FF90EF90DF90CF90BF90AF903D
:1029E000089510E09BCF7E010894E11CF11CC70103
:1029F0000E949F1F85E992E00E94B11FF60182812B
:102A00008823E1F2883008F03FC010E0198282305C
:102A100038F201E081EBA82E80E0B82E2FC0A12F64
:102A2000B0E01F5F8DB79EB708970FB6F8949EBFB2
:102A30000FBE8DBF2DB73EB72F5F3F4FEDB7FEB72F
:102A4000F282E182F901B382A282F582E482AC0DC6
:102A5000BD1DFD018485F901868317820E94022233
:102A60000F5F8DB79EB708960FB6F8949EBF0FBE46
:102A70008DBFF6018281081708F092CF183079F6E1
:102A8000A0E0B0E011E0CECFF60113811F5FBECF12
:102A9000E199FECFE199FECF20E030E03FBB2EBBB5
:102AA000E09A8DB38F3F09F41FC1E199FECFE19900
:102AB000FECF21E030E03FBB2EBBE09A8DB38F3FCD
:102AC00009F41EC1E199FECFE199FECF22E030E08A
:102AD0003FBB2EBBE09A8DB38F3F09F41CC1E19937
:102AE000FECFE199FECF23E030E03FBB2EBBE09A62
:102AF0008DB38F3F09F41AC1E199FECFE199FECF62
:102B000024E030E03FBB2EBBE09A8DB38F3F09F449
:102B100018C1E199FECFE199FECF25E030E03FBB3F
:102B20002EBBE09A8DB38F3F09F416C1E199FECF19
:102B3000E199FECF26E030E03FBB2EBBE09A8DB39B
:102B40008F3F09F414C1E199FECFE199FECF28E04F
:102B500030E03FBB2EBBE09A8DB38F3F09F413C129
:102B6000E199FECFE199FECF29E030E03FBB2EBBDB
:102B7000E09A8DB38F3F09F412C1E199FECFE1993C
:102B8000FECF2AE030E03FBB2EBBE09A8DB38F3FF3
:102B900009F411C1E199FECFE199FECF2BE030E0BD
:102BA0003FBB2EBBE09A8DB38F3F09F410C1E19972
:102BB000FECFE199FECF2CE030E03FBB2EBBE09A88
:102BC0008DB38F3F09F40FC1E199FECFE199FECF9C
:102BD0002DE030E03FBB2EBBE09A8DB38F3F09F470
:102BE0000EC1E199FECFE199FECF2EE030E03FBB70
:102BF0002EBBE09A8DB38F3F09F40DC1E199FECF52
:102C0000E199FECF2FE030E03FBB2EBBE09A8DB3C1
:102C10008F3F09F40CC1E199FECFE199FECF20E18D
:102C200030E03FBB2EBBE09A8DB38F3F09F40BC160
:102C3000E199FECFE199FECF21E130E03FBB2EBB11
:102C4000E09A8DB38F3F09F40AC1E199FECFE19973
:102C5000FECF22E130E03FBB2EBBE09A8DB38F3F29
:102C600009F409C1E199FECFE199FECF23E130E0FB
:102C70003FBB2EBBE09A8DB38F3F09F408C1E199A9
:102C8000FECFE199FECF24E130E03FBB2EBBE09ABE
:102C90008DB38F3F09F407C1E199FECFE199FECFD3
:102CA00025E130E03FBB2EBBE09A8DB38F3F09F4A6
:102CB00006C1E199FECFE199FECF26E130E03FBBAE
:102CC0002EBBE09A8DB38F3F09F405C1E199FECF89
:102CD000E199FECF27E130E03FBB2EBBE09A8DB3F8
:102CE0008F3F09F404C10895E199FECF3FBB2EBB8D
:102CF00081E08DBB0FB6F894E29AE19A0FBED5CE73
:102D0000E199FECF3FBB2EBB1DBA0FB6F894E29AF5
:102D1000E19A0FBED7CEE199FECF3FBB2EBB1DBAC5
:102D20000FB6F894E29AE19A0FBED9CEE199FECFA0
:102D30003FBB2EBB1DBA0FB6F894E29AE19A0FBEC4
:102D4000DBCEE199FECF3FBB2EBB1DBA0FB6F89488
:102D5000E29AE19A0FBEDDCEE199FECF3FBB2EBBDA
:102D60001DBA0FB6F894E29AE19A0FBEDFCEE19950
:102D7000FECF3FBB2EBB80EF8DBB0FB6F894E29A1F
:102D8000E19A0FBEE0CEE199FECF3FBB2EBB8DE7AF
:102D90008DBB0FB6F894E29AE19A0FBEE1CEE199AD
:102DA000FECF3FBB2EBB86E98DBB0FB6F894E29AEF
:102DB000E19A0FBEE2CEE199FECF3FBB2EBB8AE087
:102DC0008DBB0FB6F894E29AE19A0FBEE3CEE1997B
:102DD000FECF3FBB2EBB85E58DBB0FB6F894E29AC4
:102DE000E19A0FBEE4CEE199FECF3FBB2EBB8FEA46
:102DF0008DBB0FB6F894E29AE19A0FBEE5CEE19949
:102E0000FECF3FBB2EBB8AE58DBB0FB6F894E29A8E
:102E1000E19A0FBEE6CEE199FECF3FBB2EBB8AE022
:102E20008DBB0FB6F894E29AE19A0FBEE7CEE19916
:102E3000FECF3FBB2EBB80E58DBB0FB6F894E29A68
:102E4000E19A0FBEE8CEE199FECF3FBB2EBB88EEE4
:102E50008DBB0FB6F894E29AE19A0FBEE9CEE199E4
:102E6000FECF3FBB2EBB8CE88DBB0FB6F894E29A29
:102E7000E19A0FBEEACEE199FECF3FBB2EBB84E1C3
:102E80008DBB0FB6F894E29AE19A0FBEEBCEE199B2
:102E9000FECF3FBB2EBB84E68DBB0FB6F894E29A03
:102EA000E19A0FBEECCEE199FECF3FBB2EBB88EE80
:102EB0008DBB0FB6F894E29AE19A0FBEEDCEE19980
:102EC000FECF3FBB2EBB88E28DBB0FB6F894E29AD3
:102ED000E19A0FBEEECEE199FECF3FBB2EBB81E063
:102EE0008DBB0FB6F894E29AE19A0FBEEFCEE1994E
:102EF000FECF3FBB2EBB80E58DBB0FB6F894E29AA8
:102F0000E19A0FBE089588EC90E0089582E090E089
:102F10000895E199FECF83E090E09FBB8EBBE09ADD
:102F20008DB30895282FE199FECF83E090E09FBBF9
:102F30008EBB2DBB0FB6F894E29AE19A0FBE0895AE
:102F4000E199FECF84E090E09FBB8EBBE09A8DB309
:102F50000895282FE199FECF84E090E09FBB8EBBBF
:102F60002DBB0FB6F894E29AE19A0FBE0895E1994D
:102F7000FECF86E090E09FBB8EBBE09A8DB30895B4
:102F8000282FE199FECF86E090E09FBB8EBB2DBB42
:102F90000FB6F894E29AE19A0FBE0895E199FECF38
:102FA00087E090E09FBB8EBBE09A8DB30895282FF9
:102FB000E199FECF87E090E09FBB8EBB2DBB0FB6A3
:102FC000F894E29AE19A0FBE0895E199FECF85E068
:102FD00090E09FBB8EBBE09A8DB30895282FE199B6
:102FE000FECF85E090E09FBB8EBB2DBB0FB6F89463
:102FF000E29AE19A0FBE0895E199FECF88E090E051
:103000009FBB8EBBE09A8DB30895E199FECF89E016
:1030100090E09FBB8EBBE09A8DB30895E199FECFFF
:103020008AE090E09FBB8EBBE09A8DB30895E19952
:10303000FECF8BE090E09FBB8EBBE09A8DB30895EE
:10304000282FE199FECF88E090E09FBB8EBB2DBB7F
:103050000FB6F894E29AE19A0FBE0895282FE199ED
:10306000FECF89E090E09FBB8EBB2DBB0FB6F894DE
:10307000E29AE19A0FBE0895282FE199FECF8AE0E7
:1030800090E09FBB8EBB2DBB0FB6F894E29AE19AFD
:103090000FBE0895282FE199FECF8BE090E09FBBF3
:1030A0008EBB2DBB0FB6F894E29AE19A0FBE08953D
:1030B000E199FECF8CE090E09FBB8EBBE09A8DB390
:1030C0000895E199FECF8DE090E09FBB8EBBE09A22
:1030D0008DB30895E199FECF8EE090E09FBB8EBB4B
:1030E000E09A8DB30895E199FECF8FE090E09FBB09
:1030F0008EBBE09A8DB30895282FE199FECF8CE026
:1031000090E09FBB8EBB2DBB0FB6F894E29AE19A7C
:103110000FBE0895282FE199FECF8DE090E09FBB70
:103120008EBB2DBB0FB6F894E29AE19A0FBE0895BC
:10313000282FE199FECF8EE090E09FBB8EBB2DBB88
:103140000FB6F894E29AE19A0FBE0895282FE199FC
:10315000FECF8FE090E09FBB8EBB2DBB0FB6F894E7
:10316000E29AE19A0FBE0895E199FECF84E190E0E2
:103170009FBB8EBBE09A8DB30895E199FECF85E1A8
:1031800090E09FBB8EBBE09A8DB30895E199FECF8E
:1031900086E190E09FBB8EBBE09A8DB30895E199E4
:1031A000FECF87E190E09FBB8EBBE09A8DB3089580
:1031B000282FE199FECF84E190E09FBB8EBB2DBB11
:1031C0000FB6F894E29AE19A0FBE0895282FE1997C
:1031D000FECF85E190E09FBB8EBB2DBB0FB6F89470
:1031E000E29AE19A0FBE0895282FE199FECF86E179
:1031F00090E09FBB8EBB2DBB0FB6F894E29AE19A8C
:103200000FBE0895282FE199FECF87E190E09FBB84
:103210008EBB2DBB0FB6F894E29AE19A0FBE0895CB
:10322000E199FECF80E190E09FBB8EBBE09A8DB329
:103230000895E199FECF81E190E09FBB8EBBE09ABB
:103240008DB30895E199FECF82E190E09FBB8EBBE4
:10325000E09A8DB30895E199FECF83E190E09FBBA2
:103260008EBBE09A8DB30895282FE199FECF80E1BF
:1032700090E09FBB8EBB2DBB0FB6F894E29AE19A0B
:103280000FBE0895282FE199FECF81E190E09FBB0A
:103290008EBB2DBB0FB6F894E29AE19A0FBE08954B
:1032A000282FE199FECF82E190E09FBB8EBB2DBB22
:1032B0000FB6F894E29AE19A0FBE0895282FE1998B
:1032C000FECF83E190E09FBB8EBB2DBB0FB6F89481
:1032D000E29AE19A0FBE089588E192E090936A0223
:1032E000809369021092180208958F929F92AF9274
:1032F000BF92DF92EF92FF920F931F93DF93CF93D2
:10330000CDB7DEB76E970FB6F894DEBF0FBECDBF58
:103310004E010894811C911CC40161E976E04AE0E9
:1033200050E00E94DC216A817B8161157105E9F121
:10333000DD248BE0A82EB12CAC0EBD1EC5010E9471
:10334000E52189859A85892BF9F08A819B810E94E4
:10335000B11F89E797E00E94B11FE985FA850995B9
:10336000E82EFF2400E010E08AE063E040E020E285
:103370000E94D51F85E797E00E94B11F8C819D8137
:103380000E94B11F0E94C81FD3946AE0D69EB0016C
:1033900011246F56794FC4014AE050E00E94DC21AD
:1033A0006A817B816115710549F682E493E00E9490
:1033B000B11F81E797E00E94B11F0E94B71787FDF8
:1033C0002EC085958595E82EFF24E7FCF094002714
:1033D000F7FC0095102F8AE064E041E020E20E94B3
:1033E000D51F8DE697E00E94B11F83EC95E00E9407
:1033F000B11F0E94C81F80E090E06E960FB6F8944F
:10340000DEBF0FBECDBFCF91DF911F910F91FF9017
:10341000EF90DF90BF90AF909F908F9008958D5F59
:10342000D0CFEF92FF920F931F93FC0180818823EE
:10343000E9F40E94B71787FD27C085958595E82E8A
:10344000FF24E7FCF0940027F7FC0095102F8AE09A
:1034500064E041E020E20E94D51F0E94C81F80E086
:1034600090E01F910F91FF90EF900895CF010E947F
:10347000BE21880F880F0E94C01780E090E01F9146
:103480000F91FF90EF9008958D5FD7CFEF92FF924D
:103490000F931F93FC0180818823A9F40E94CF1809
:1034A000E82EFF2400E010E08AE063E040E020E244
:1034B0000E94D51F0E94C81F80E090E01F910F91CD
:1034C000FF90EF900895CF010E94BE210E94021943
:1034D00080E090E01F910F91FF90EF900895EF92A0
:1034E000FF920F931F93FC0180818823A9F40E940F
:1034F000BD18E82EFF2400E010E08AE063E040E021
:1035000020E20E94D51F0E94C81F80E090E01F911A
:103510000F91FF90EF900895CF010E94BE210E946D
:10352000E61880E090E01F910F91FF90EF900895D2
:10353000EF92FF920F931F93FC0180818823A9F4DF
:103540000E94B418E82EFF2400E010E08AE063E057
:1035500040E020E20E94D51F0E94C81F80E090E05A
:103560001F910F91FF90EF900895CF010E94BE210F
:103570000E94D81880E090E01F910F91FF90EF908B
:103580000895EF92FF920F931F93FC01808188238F
:10359000A9F40E942B19E82EFF2400E010E08AE035
:1035A00063E040E020E20E94D51F0E94C81F80E037
:1035B00090E01F910F91FF90EF900895CF010E942E
:1035C000BE210E945E1980E090E01F910F91FF9054
:1035D000EF900895EF92FF920F931F93FC0180816B
:1035E0008823A9F40E941919E82EFF2400E010E0B6
:1035F0008AE063E040E020E20E94D51F0E94C81FDD
:1036000080E090E01F910F91FF90EF900895CF011F
:103610000E94BE210E94421980E090E01F910F910C
:10362000FF90EF900895EF92FF920F931F93FC018C
:1036300080818823A9F40E941019E82EFF2400E05D
:1036400010E08AE063E040E020E20E94D51F0E9483
:10365000C81F80E090E01F910F91FF90EF900895B8
:10366000CF010E94BE210E94341980E090E01F919A
:103670000F91FF90EF900895EF92FF920F931F9399
:10368000FC0180818823A9F40E947318E82EFF248E
:1036900000E010E08AE063E040E020E20E94D51FF5
:1036A0000E94C81F80E090E01F910F91FF90EF9063
:1036B0000895CF010E94BE210E94A61880E090E0EC
:1036C0001F910F91FF90EF900895EF92FF920F934B
:1036D0001F93FC0180818823A9F40E946118E82EC1
:1036E000FF2400E010E08AE063E040E020E20E9476
:1036F000D51F0E94C81F80E090E01F910F91FF909E
:10370000EF900895CF010E94BE210E948A1880E0A8
:1037100090E01F910F91FF90EF900895EF92FF922C
:103720000F931F93FC0180818823A9F40E945818ED
:10373000E82EFF2400E010E08AE063E040E020E2B1
:103740000E94D51F0E94C81F80E090E01F910F913A
:10375000FF90EF900895CF010E94BE210E947C1837
:1037600080E090E01F910F91FF90EF900895EF920D
:10377000FF920F931F93FC0180818823A9F40E947C
:103780001718E82EFF2400E010E08AE063E040E034
:1037900020E20E94D51F0E94C81F80E090E01F9188
:1037A0000F91FF90EF900895CF010E94BE210E94DB
:1037B0004A1880E090E01F910F91FF90EF900895DC
:1037C000EF92FF920F931F93FC0180818823A9F44D
:1037D0000E940518E82EFF2400E010E08AE063E074
:1037E00040E020E20E94D51F0E94C81F80E090E0C8
:1037F0001F910F91FF90EF900895CF010E94BE217D
:103800000E942E1880E090E01F910F91FF90EF90A2
:103810000895EF92FF920F931F93FC0180818823FC
:10382000A9F40E94FC17E82EFF2400E010E08AE0D3
:1038300063E040E020E20E94D51F0E94C81F80E0A4
:1038400090E01F910F91FF90EF900895CF010E949B
:10385000BE210E94201880E090E01F910F91FF9000
:10386000EF900895EF92FF920F931F9380E00E94D4
:10387000DA1D7C0183E897E00E94B11FF694E7947B
:10388000F694E79400E010E08AE064E041E020E292
:103890000E94D51F8DE797E00E94B11F0E94C81FAC
:1038A00080E090E01F910F91FF90EF9008950F93AB
:1038B0001F938C010E94BE210E949217C8010E9492
:1038C000BE21892B59F48BE897E00E94B11F0E941A
:1038D000C81F80E090E01F910F91089587E997E05D
:1038E0000E94B11F0E94C81F80E090E01F910F91BD
:1038F00008950F931F938C010E94BE210E94A91767
:10390000C8010E94BE21892B59F482EA97E00E94E7
:10391000B11F0E94C81F80E090E01F910F91089591
:103920008EEA97E00E94B11F0E94C81F80E090E0DD
:103930001F910F9108950F931F938C010E94BE2138
:103940000E94EE17C8010E94BE21892B31F489EB39
:1039500097E00E94B11F0E94C81F80E090E01F9175
:103960000F91089585EE95E00E94B11F0E94CE1739
:103970008F3F29F00E94C81F80E090E008958AE3FD
:1039800096E00E94B11F0E94C81F80E090E0089559
:103990001F938CEC97E00E94B11F0E94C81F1092E9
:1039A000A9018FE991E061E976E04AE050E00E94E8
:1039B000DC218091A0019091A101009729F11AE0EA
:1039C0000E94B11F88EC97E00E94B11F8091A20174
:1039D0009091A3010E94B11F0E94C81F6091A9018C
:1039E0006F5F6093A901619FB00111246F56794FF9
:1039F0008FE991E04AE050E00E94DC218091A00133
:103A00009091A1010097E1F60E94CE178F3F21F01F
:103A100080E090E01F9108958AE396E00E94B11F34
:103A200080E090E01F910895DF92EF92FF920F9354
:103A30001F93DF93CF93CDB7DEB764970FB6F8949B
:103A4000DEBF0FBECDBF1092B4018AEA91E061E9FA
:103A500076E04AE050E00E94DC216091AB01709179
:103A6000AC0161157105E9F17E010894E11CF11CBE
:103A70002AE0D22E17C06091B4016F5F6093B40149
:103A80006D9DB00111246F56794F8AEA91E04AE0AA
:103A900050E00E94DC216091AB017091AC01611596
:103AA0007105F9F0C7010E94E521F701019000209E
:103AB000E9F78F01015010400E191F09C70168E195
:103AC00072E0A8010E94EC210097A9F6E091B001F4
:103AD000F091B101309789F0C801885E9D4F09953A
:103AE0000CC088EE97E00E94B11F0E94C81F8BEDAA
:103AF00097E00E94B11F0E94C81F64960FB6F89409
:103B0000DEBF0FBECDBFCF91DF911F910F91FF9010
:103B1000EF90DF9008951F93182F0E94991F1A307D
:103B200059F11D3049F11830B1F0E0916902F0917E
:103B30006A0282E0E836F80760F41083E0916902D7
:103B4000F0916A023196F0936A02E093690231972C
:103B500011821F910895E0916902F0916A0222E0BA
:103B6000E831F207B1F3A8F33197F0936A02E093DA
:103B7000690210821F9108958091690290916A02F2
:103B80008851924031F328F30E94C81F0E94141DEF
:103B900088E192E090936A02809369021092180281
:103BA0001F910895A19884B3816484BBA898AE9AAC
:103BB000A9980895CF93DF93A898AE98A89A83B355
:103BC00090E0A898A89A8270907099990196A89808
:103BD000A89A880F991F99990196A898A89A880F72
:103BE000991F99990196A898A89A880F991F999951
:103BF0000196A898A89A880F991F99990196A89854
:103C0000A89A880F991F99990196A898A89A880F41
:103C1000991F99990196A898A89A880F991F999920
:103C20000196A898A89A880F991F99990196A89823
:103C3000A89A880F991F99990196A898A89A880F11
:103C4000991F99990196A898A89AEC01CC0FDD1FAD
:103C500099992196A898A89A0E94B7178F3F39F092
:103C60000E94B717992787FD9095C80FD91F99997A
:103C70000AC0A898A89AA898A89AA898AE9ACE011F
:103C8000DF91CF910895CFEFDFEFF3CFFC01718388
:103C900060835383428317821682158214820895AB
:103CA000CF93DF93EC012C813D8121153105E1F0AB
:103CB0008E819F81E881F981E80FF91FE0810196EB
:103CC0009F838E836A817B818617970740F42150FA
:103CD00030403D832C838E2FDF91CF9108950E9439
:103CE000C2249F838E83F3CFE0E08E2FDF91CF91AC
:103CF0000895CF93DF93FC01EB0124813581621796
:103D00007307B0F486819781860F971F9783868308
:103D1000628173818617970720F00E94C2249783DF
:103D200086832C1B3D0B35832483DF91CF9108952F
:103D300015821482DF91CF910895FC01CB01268179
:103D4000378162817381820F931F0E94C224019088
:103D5000F081E02DE80FF91F80810895CF93DF9364
:103D6000EC01462F2C813D813093B6012093B501A3
:103D70006A817B8126173707A0F48E819F81820F8D
:103D8000931F0E94C224E881F981E80FF91F408344
:103D90008C819D8101969D838C838FEFDF91CF91E4
:103DA000089580E0DF91CF910895FC0140E02481E7
:103DB0003581828193812817390708F441E0842FE7
:103DC0000895FC0140E084819581860F971F228130
:103DD00033818217930708F441E0842F0895FC0192
:103DE00084810895FC011582148208950F931F9316
:103DF000CF93DF93EC018B01FB014081442309F158
:103E00002C813D813093B6012093B5016A817B817D
:103E10002617370780F48E819F81820F931F0E949F
:103E2000C224E881F981E80FF91F40838C819D81CC
:103E300001969D838C830F5F1F4FF80140814423BF
:103E4000F9F68FEFDF91CF911F910F91089585368D
:103E500038F48093BA018093BB01882329F0089538
:103E60001092BA011092BB01E0916C02F0916D02C8
:103E7000908180916B02809589238083C59A0895F3
:103E8000E0916C02F0916D02908180916B028095BF
:103E900089238083C59A1092BA0108958091BB014D
:103EA0008093BA0108952091BA01222319F18091DB
:103EB000B9018F5F8093B901853678F081E08093F6
:103EC000B901E0916C02F0916D02808190916B02DA
:103ED000892B8083C5988091B901281758F4E09107
:103EE0006C02F0916D02908180916B028095892324
:103EF0008083C59A089570936D0260936C0240931D
:103F00006B021092B9011092BA011092BB019AE0B3
:103F1000899FB001112483E59FE10E94170D9093C2
:103F2000B8018093B70108959093BD018093BC01BF
:103F30000895E091BC01F091BD0109950895CF93DA
:103F4000DF93EC01009739F409C02196E091BC01A0
:103F5000F091BD01099588818823B9F7DF91CF9150
:103F60000895CF93DF93FC01009779F08491882323
:103F700061F0EF012196E091BC01F091BD0109953E
:103F8000FE01219684918823B1F7DF91CF910895A6
:103F9000E091BC01F091BD018DE00995E091BC017B
:103FA000F091BD018AE0099508952F923F924F92BA
:103FB0005F926F927F928F929F92AF92BF92CF92B9
:103FC000DF92EF92FF920F931F93DF93CF93CDB7C2
:103FD000DEB7A4970FB6F894DEBF0FBECDBF6AA3BD
:103FE0004BA32CA317012801442311F017FD92C005
:103FF00082017101AAA0AA9490E02BA1211191E065
:10400000AA2DA91BA9A318A2682E77248824992475
:10401000C801B701A40193010E94E924FB01E45007
:10402000F84F64916F8FC801B701A40193010E94FA
:10403000E924C901DA017C018D018EE1C82ED12C61
:10404000CC0EDD1EB9A01AC0C801B701A4019301AE
:104050000E94E924FB01E450F84F6491F60160836B
:10406000C801B701A40193010E94E924C901DA0142
:104070007C018D01BA940894C108D108BB2049F095
:10408000E114F10401051105F9F6ECA1D601EC9358
:10409000F1CFCE014F968C01F9A10F1B11092BA175
:1040A000222359F057FC31C021143104410451043A
:1040B000C9F18BE2F80182938F01BAA1BB2311F4FD
:1040C0000BC0AA94E091BC01F091BD01D8018D9183
:1040D0008D010995AA20A9F7A4960FB6F894DEBF22
:1040E0000FBECDBFCF91DF911F910F91FF90EF9049
:1040F000DF90CF90BF90AF909F908F907F906F9008
:104100005F904F903F902F9008958DE2D8018E934D
:104110008D01D3CFEE24FF248701E218F3080409B0
:10412000150968CF80E2D8018E938D01C6CF909398
:104130000F0280930E0208959B01AC016050704FF6
:10414000814F9F4F660F771F881F991F660F771F3C
:10415000881F991F660F771F881F991F220F331F13
:10416000441F551F220F331F441F551F220F331F9B
:10417000441F551F220F331F441F551F0E94E9245F
:10418000215029B908958FE692E0089588E792E0DA
:104190000895982F80916E028823E1F39CB91092C4
:1041A0006E020895982F80916E028823E1F39CB9E6
:1041B00010926E0281E090E00895109274021092C5
:1041C0007302089520E08091730290917402892B0C
:1041D00009F421E0822F08951F920F920FB60F92DB
:1041E00011242F933F934F935F936F937F938F93FC
:1041F0009F93AF93BF93EF93FF936CB18FE692E0E1
:104200000E94AE1EFF91EF91BF91AF919F918F9150
:104210007F916F915F914F913F912F910F900FBEC2
:104220000F901F901895682F88E792E00E94AE1EAD
:1042300008951F920F920FB60F9211242F933F9360
:104240004F935F936F937F938F939F93AF93BF939E
:10425000EF93FF9380917702882361F080917C0235
:1042600090917D02892BD1F41092770281E08093A6
:104270006E0203C081E080936E02FF91EF91BF91C7
:10428000AF919F918F917F916F915F914F913F91EE
:104290002F910F900FBE0F901F90189588E792E016
:1042A0000E94501E8CB9E9CF80917C0290917D02D2
:1042B000892B19F0809177028111089581E0809314
:1042C000770288E792E00E94501E982F80916E023C
:1042D0008823E1F39CB910926E020895CF93DF9387
:1042E000EC018091710290917202892B31F08091E2
:1042F000730290917402892B21F480E0DF91CF91B9
:1043000008958FE692E00E94501E888381E0DF913D
:10431000CF9108958FE692E06EEB71E048E250E0B5
:104320000E94461E88E792E066EE71E048E250E0A7
:104330000E94461E08958FE692E06EEB71E048E21F
:1043400050E00E94461E88E792E066EE71E048E287
:1043500050E00E94461E10920F0210920E0288ED4D
:104360008AB98FE289B981E080936E021092770258
:10437000109281021092800278940895FC0188279F
:104380009927E89421912032E9F3293010F02E305A
:10439000C8F32B3241F02D3239F4689404C00E94E6
:1043A000FA21820F911D219120532A30C0F31EF46F
:1043B000909581959F4F0895FB01DC0102C0059007
:1043C0000D9241505040D8F70895FB01DC01059053
:1043D0000D920020E1F70895FB01DC0141505040AF
:1043E00030F08D910190801919F40020B9F7881BE5
:1043F000990B08957AE0979F902D879F802D910DBE
:1044000011240895AEE0B0E0E8E0F2E20C94342527
:104410000D891E8986E08C831A8309838FEF9FE7BD
:104420009E838D839E01275E3F4FCE0101966F894B
:10443000788DA9010E9426222F813885020F131F33
:10444000F80110822E96E4E00C945025ABE0B0E029
:10445000ECE2F2E20C9426253C012B015A01FC010E
:1044600017821682838181FD03C06FEF7FEFC6C183
:104470009AE0892E1E010894211C311CF30123812E
:10448000F20123FD859123FF81912F01882309F4F7
:10449000B2C1853239F423FD859123FF81912F012B
:1044A000853229F490E0B3010E941924E7CF982FB8
:1044B000FF24EE249924FFE1FF15D0F09B3269F030
:1044C0009C3228F4903259F0933291F40EC09D3210
:1044D00049F0903369F441E024C052E0F52A84E0C9
:1044E000F82A28C098E0F92A25C0E0E1FE2A22C077
:1044F000F7FC29C0892F80538A3070F4F6FE05C07E
:10450000989C902C1124980E15C0E89CE02C112446
:10451000E80EF0E2FF2A0EC09E3229F4F6FC6BC1D1
:1045200040E4F42A07C09C3619F450E8F52A02C08A
:10453000983649F4F20123FD959123FF91912F01C3
:10454000992309F0B8CF892F8554833018F0805211
:10455000833038F444E050E0A40EB51E5FE3598385
:104560000FC0933631F0933779F0933509F056C088
:1045700020C0F5018081898342E050E0A40EB51E81
:10458000610101E010E012C0F501C080D180F6FCAD
:1045900003C06FEF7FEF02C0692D70E042E050E092
:1045A000A40EB51EC6010E940E248C015FE7F52201
:1045B00014C0F501C080D180F6FC03C06FEF7FEF1F
:1045C00002C0692D70E042E050E0A40EB51EC601A5
:1045D0000E9403248C0150E8F52AF3FE07C01AC09C
:1045E00080E290E0B3010E941924EA948E2D90E0BD
:1045F00008171907A8F30EC0F601F7FC8591F7FE1E
:1046000081916F0190E0B3010E941924E110EA94B6
:10461000015010400115110579F7EAC0943611F0E8
:10462000993669F5F7FE08C0F50120813181428194
:10463000538184E090E00AC0F501808191819C0162
:10464000442737FD4095542F82E090E0A80EB91E14
:104650009FE6F92257FF09C0509540953095219566
:104660003F4F4F4F5F4FE0E8FE2ACA01B901A10159
:104670002AE030E00E944524D82ED21840C0953759
:1046800029F41F2D1F7E2AE030E01DC01F2D197F49
:104690009F3661F0903720F4983509F0ACC00FC018
:1046A000903739F0983709F0A6C004C028E030E010
:1046B0000AC0106114FD146020E130E004C014FD54
:1046C000166020E132E017FF08C0F50160817181BA
:1046D0008281938144E050E008C0F501808191819E
:1046E000BC0180E090E042E050E0A40EB51EA101C4
:1046F0000E944524D82ED2188FE7F82EF122F6FE1C
:104700000BC05EEFF522D91438F4F4FE07C0F2FCBA
:1047100005C08FEEF82202C01D2D01C0192DF4FE38
:104720000DC0FE01ED0DF11D8081803319F499EE6D
:10473000F92208C01F5FF2FE05C003C08F2D8678E6
:1047400009F01F5F0F2DF3FC14C0F0FE0FC01E1503
:1047500010F09D2C0BC09D2C9E0C911A1E2D06C096
:1047600080E290E0B3010E9419241F5F1E15C0F380
:1047700004C01E1510F4E11A01C0EE2404FF0FC09E
:1047800080E390E0B3010E94192402FF1DC001FDE7
:1047900003C088E790E00EC088E590E00BC0802F52
:1047A000867891F001FF02C08BE201C080E2F7FC45
:1047B0008DE290E0B3010E94192406C080E390E0EE
:1047C000B3010E9419249A94D914C0F3DA94F10128
:1047D000ED0DF11D808190E0B3010E941924DD20D0
:1047E000A9F706C080E290E0B3010E941924EA9480
:1047F000EE20C1F743CEF30166817781CB012B9682
:10480000E2E10C944225FC010590615070400110DA
:10481000D8F7809590958E0F9F1F0895FC016150E9
:10482000704001900110D8F7809590958E0F9F1FD2
:1048300008950F931F93CF93DF938C01EB018B812E
:1048400081FF1BC082FF0DC02E813F818C819D8125
:104850002817390764F4E881F9810193F983E88323
:1048600006C0E885F985802F0995892B31F48E8162
:104870009F8101969F838E8302C00FEF1FEFC801B7
:10488000DF91CF911F910F910895FA01AA27283047
:1048900051F1203181F1E8946F936E7F6E5F7F4F0D
:1048A0008F4F9F4FAF4FB1E03ED0B4E03CD0670F89
:1048B000781F891F9A1FA11D680F791F8A1F911DDC
:1048C000A11D6A0F711D811D911DA11D20D009F42C
:1048D00068943F912AE0269F11243019305D31936E
:1048E000DEF6CF010895462F4770405D4193B3E057
:1048F0000FD0C9F7F6CF462F4F70405D4A3318F0FE
:10490000495D31FD4052419302D0A9F7EACFB4E0AE
:10491000A6959795879577956795BA95C9F7009766
:104920006105710508959B01AC010A2E0694579507
:10493000479537952795BA95C9F7620F731F841F5E
:10494000951FA01D0895629FD001739FF001829F63
:10495000E00DF11D649FE00DF11D929FF00D839F0E
:10496000F00D749FF00D659FF00D9927729FB00DAB
:10497000E11DF91F639FB00DE11DF91FBD01CF01BE
:1049800011240895AA1BBB1B51E107C0AA1FBB1F1E
:10499000A617B70710F0A61BB70B881F991F5A95CB
:1049A000A9F780959095BC01CD01089597FB092E3C
:1049B00007260AD077FD04D0E5DF06D000201AF4E0
:1049C000709561957F4F0895F6F7909581959F4F6B
:1049D0000895A1E21A2EAA1BBB1BFD010DC0AA1F40
:1049E000BB1FEE1FFF1FA217B307E407F50720F058
:1049F000A21BB30BE40BF50B661F771F881F991FD3
:104A00001A9469F760957095809590959B01AC011B
:104A1000BD01CF01089597FB092E05260ED057FD45
:104A200004D0D7DF0AD0001C38F45095409530955B
:104A300021953F4F4F4F5F4F0895F6F79095809522
:104A4000709561957F4F8F4F9F4F08952F923F92A2
:104A50004F925F926F927F928F929F92AF92BF928E
:104A6000CF92DF92EF92FF920F931F93CF93DF933A
:104A7000CDB7DEB7CA1BDB0B0FB6F894DEBF0FBE97
:104A8000CDBF09942A88398848885F846E847D84E4
:104A90008C849B84AA84B984C884DF80EE80FD80E6
:104AA0000C811B81AA81B981CE0FD11D0FB6F8945C
:0E4AB000DEBF0FBECDBFED010895F894FFCF1D
:104ABE00AE01B501C701CE01D701DE01E701EE015E
:104ACE00FA0101020A0211021A02210224022B0229
:104ADE00310238023E0245024E0255025E02650266
:104AEE006E0275027E0285020000000000FE0001CB
:104AFE000601020A01031401041F010525010037F6
:0A4B0E0001257320253032640000F9
:00000001FF
